:030000000219FDE5
:03000B000200AA46
:03002B0002015F70
:03005B000202E7B7
:030073000202CDB9
:1000800002030406080C10182030406080040608A3
:100090000C10182030406080A0C000070F1F3F0DDB
:1000A0000D04050D050205030302C2AFC0D0C0E078
:1000B000206217E5256002E473E525F4F58A758B67
:1000C00000D262D0E0D0D0D2AF3285268AC262E5BB
:1000D00026F4602F758B00D0E0D0D0D290D291D290
:1000E00092D2AF32D290D291D292206E0C20660979
:1000F000740AD5E0FDE57E4290758B00D0E0D0D04B
:10010000D2AF32758A00C28DD26201F901B930686E
:1001100005206602C29001B9306805206602C291CE
:1001200001B9306805206602C29201B9C2933068F5
:100130000A2066077428D5E0FDC29001B9C2943048
:10014000680A2066077428D5E0FDC29101B9C295FE
:1001500030680A2066077428D5E0FDC29201B9C252
:10016000AFC2AD53E6EFC0D0C0E0D2D3D2AFC2CE63
:10017000E52A6007207449152A21C07800790020FB
:10018000742EE580307E01F430E70278FF53DACF39
:10019000207E0343DA20307E0343DA10C2D8C271D6
:1001A000E580307E01F430E70279FFC3E89970CB37
:1001B000306103752A18207403752A18885FD2707D
:1001C00020740DE52B6004152B21D043DA01C2D831
:1001D000207002412EA85F206102C270207436791F
:1001E00082B70431C3E894F0400374F0F8E8C454D3
:1001F0000F28F87984B703024115C313C31387216D
:10020000200802C313200A06C3C898F8411528F82D
:10021000500374FFF88822E52D54066011E533C3BE
:1002200013C31324062522F52250037522FF78827A
:10023000B6044E852224A824C3E52495644002A870
:1002400064C3E895664002A8668825E569700241A6
:100250007FC3E8AA699A5003E8FAE4F9EAC333FBDA
:10026000E56BF45B29400D256AF8E56A6002156AC2
:10027000400B417F0AC3E56A9A5002056A78FF88FD
:1002800026C3E52594404002D26420CF0AD0E0D0B6
:10029000D043E610D2AD32C2CF053A7801E52A60EC
:1002A00005307402152AC3E55F94014005756200AC
:1002B00041C3756300756C00E5622401F56250036B
:1002C0007562FFD0E0D0D043E610D2AD32C2AFC0ED
:1002D000D053E67FC2607591008556948557957519
:1002E0009104D0D0D2AF32C2AF53E6EFC2ADC0D08E
:1002F000C0E0C0F0D2D3D2AFA8FBA9FCC2D8307105
:1003000002614E53DACF207E0343DA10307E03437E
:10031000DA20D271E580307E01F420E70261258881
:10032000278928A17B53DACF207E0343DA20307E51
:100330000343DA10C2D8C271307402A1677800E5B5
:1003400080307E01F430E702A167885FA14F53DA65
:10035000CF207E0343DA20307E0343DA10C27120BF
:100360006102812753DACF207E0343DA10307E0307
:1003700043DA20C2D8D271885A895BC3E89558F80D
:10038000E99559F97B007E087A00C3E8948CE994DA
:10039000005005755E008119882178A2E6A82160C9
:1003A00055C3E894C8E994005008E4D2E4FB7A0A03
:1003B00061F4C3E89468E994015008E4D2E3FB7A5D
:1003C0000F61F4C3E894D0E994025008E4D2E2FB50
:1003D0007A1E61F4C3E894A0E994055008E4D2E1E0
:1003E000FB7A3C61F4C3E89498E994085008E4D29D
:1003F000E0FB7A787E00C3E8955CFCE9955DFD3012
:10040000E70AECF42401FCEDF43400FD755E00C352
:10041000EC9AED9E5003755E01885C895D855A58A3
:10042000855B597802A14FC3E89527F8E99528F92B
:10043000307C02A133307B02A133307A02A12C2020
:100440007502814AE9FDE8FC8169E9C313F9E81303
:10045000F8307902A12CE9C313F9E813F8307802D7
:10046000A12CE9C313FDE813FC20612CC3EC941C00
:0E047000ED940240028180ED701EC3EC94C832
:10047E0050180529E52970021529C3E529940A505B
:10048E0002A167755F00D270A167E5296002152988
:10049E007888E6F97400207F087896B90302789E72
:1004AE00E624FAFEE43400FFC3EC9EFCED9FFD92C1
:1004BE0008B90310A2085007207609D27681D230EF
:1004CE007602C276A2085016B9030DECF42401FC94
:1004DE00EDF43400FD0204EC78007900A133B90389
:1004EE0015EC33FCED33FDC3EC940AFCED9400FDEA
:1004FE0050047C007D00C3EC94FFED940040067820
:10050E00FF7900A133EC8575F0A4C5F0A2F733F89E
:10051E007900400302054F78FF790002054FE9C3C9
:10052E0013F9E813F8307C0EE9600278FFC3E81384
:10053E0038F8E43400F9C3E894FFE99400400278F7
:10054E00FF885FD270206102A167741FF4552F4B94
:10055E00F52FC274EB7002D274752A1830740375BD
:10056E002A0A306102A17B20740353DAFE20740341
:10057E00752B06D0F0D0E0D0D0D2AD43E610327954
:10058E00010205AB79030205AB790A0205AB791EB0
:10059E000205AB79640205AB79C80205AB7817E4A6
:1005AE00D5E0FDD8FAD9F6227A147B780205D27AF4
:1005BE00107B8C0205D27A0D7BB40205D27A0B7BAE
:1005CE00C80205D27902B27DE4C294D5E0FDC29193
:1005DE00D5E0FDD291D5E0FDD294D5E0FDC290E5F7
:1005EE0076D5E0FDD2907496D5E0FDD9D9EAF8D54E
:1005FE00E0FDD8FBDBCEC29422C37C007D0075F0FB
:10060E000005F0EA33FAEB33FB50F6EB13FBEA137B
:10061E00FAC3E9FFE8FEE89AF8E99BF95004EFF90E
:10062E00EEF8B3EC33FCED33FDD5F0DFEDF9ECF87D
:10063E0022E889F08A20D2D4F8A9F07B0030F70B9B
:10064E007BFFF42401F8E9F43400F9E88520F0A4E6
:10065E00ADF0F8E98520F0A4AFF0FEED2EF97400B0
:10066E003FFA7C04C3EA13FAE913F9E813F8DCF451
:10067E008BF030F70AE8F42401F8E9F43400F9E8D5
:10068E0089F0C2D4F8A9F0227882B604030206F1EA
:10069E00C3E55F940140030206BB852224E4F545C1
:1006AE00F546F547F548F549C26D0206F17882E642
:1006BE00FCD26DE522F523783879C7AA40AB41C349
:1006CE00EB13FBEA13FAEC146013C3EB13FBEA1300
:1006DE00FAEC14146007C3EB13FBEA13FAD1078884
:1006EE0045894622C3E5459523F8E5469400F95021
:1006FE000CC3E89480E994FF4016020722C3E894E5
:10070E007FE994005003020722787F7900020722C6
:10071E00788079FF884A894B22E54A2547F8E54BD0
:10072E003548F9854B20E4300701F43549FA30E7B6
:10073E0009C3EA94F04015020760C3EA940F500310
:10074E0002076078FF79FF7A0F0207607800790060
:10075E007AF0C3E5249564500AC374019524500BB6
:10076E0002077EE54B20E70E02077EE54B30E706DB
:10077E00884789488A492278A4E6FAC3E54A33F8BD
:10078E00E54B33F9D13FE930E70BC3E89480E994A8
:10079E00FF4013E1B8C3E8947FE994005002E1B83A
:1007AE00787F7900E1B8788079FFE820E715C3E516
:1007BE002398F84009C3E8940140030207DF78014B
:1007CE000207DFE8F424012523F840030207DF784F
:1007DE00FF884C2278A5E6FAA848A949D13FE9300E
:1007EE00E70CC3E89401E994FF4016020813C3E82E
:1007FE0094FFE99400500302081378FF7900020871
:10080E0013780179FFE920E715C3E54C98F8400904
:10081E00C3E89401400302083A780102083AE8F46A
:10082E002401254CF8400302083A78FF88242278E8
:10083E00FFC26420693D206A12D264C3E541940A66
:10084E004009C3E52594405002C26479A1E76023B4
:10085E00E541601F74FF8541F0848539F0306A03ED
:0F086E0075F005A4F8C5F0600278FFC3E8956740
:10087D005002A867886622C3E5409440E541940183
:10088D00E5665003140195046002F5662202089D89
:10089D002275E890227883E6FFE5E820ECF7A8BD05
:1008AD00A9BE0573C3E57394084052757300E9FA48
:1008BD0079A0E76044EA7007E574601B0208D8C3AD
:1008CD00E895746010E5745006600C140208E40499
:1008DD0060F90208E4E574F574C3946D401B75640A
:1008ED00C0C394044013756480C39404400B7564B5
:1008FD0040C39404400375640075BB0622E564246F
:10090D0010500274FFF5647982B704022131C3A837
:10091D0064E524985002A824C3E895664002A866B1
:10092D0088258826E573B4070375BB1022743279C8
:10093D00A687F0A4C5F0A2F733F8C3E8956440028A
:10094D00A864882288248825882688672275400017
:10095D007541F022C2AF75C820A8CCA9CDAA3A30F6
:10096D00CF010A75C824D2AFAB3BAC3C883B893C68
:10097D00C3E89BF8E99C206908F9306702417621AC
:10098D00D3AD3D8A3DF9EA9DFA600478FF79FFAE5B
:10099D003EAF3F8B3E8C3FC3EC9FFCC3E99CF542C1
:1009AD00A83BA93CC3E89EF8E99FF9C3E54113FBB9
:1009BD00E54013FAE82AF540E93BF541500675404C
:1009CD00FF7541FF411DAA40AB41AC40AD417E04D6
:1009DD007F02C3EB940440021E1FC3EB9408400238
:1009ED001E1FC3ED13FDEC13FCDEF7C3EA9CFAEBFF
:1009FD009DFBEF6009C3E913F9E813F8DFF7EA2867
:100A0D00FAEB39FB8A408B4150067BFF8B408B41C3
:100A1D00C3EB94025002D2673069047F03414878DA
:100A2D0092E6FFC3E537948240110FC3E53794A0DA
:100A3D0040010FC3EF940640027F057E07E541C4D8
:100A4D00540FF9E541C454F0F8E540C4540F28F8AB
:100A5D00C3E89EFAE99400FB4009C3EA9402EB94C3
:100A6D000050047A02E4FB41C2AA40AB41EBC4FE44
:100A7D00EAC4540F4EFCC3EA9CFAEB9400FBC3E8A6
:100A8D0013C313F8EA28FAEB3400FB8A408B41C3F9
:100A9D00EB94024002C2677807EBC4FE7B00EAC408
:100AAD00540F4EFAC3EA98FA4005C3940250027AE5
:100ABD00027892E6FF30600241C285525685535747
:100ACD00D26043E680C3E49AF8E49BF93067026193
:100ADD005CE8FAE9FBD3E913FDE813FC885289536E
:100AED00C3EF94036038EF20E00DE82CF8E93DF9F1
:100AFD00ECFAEDFB020B17E828F8E939F9C3E82405
:100B0D0002F8E93400F97AFE7BFFC3EF9403400E3F
:100B1D008A548B55884E894F8C508D5161908854D5
:100B2D0089558A4E8B4F8C508D51306920C3E533DA
:100B3D0094034019E542A2E713F8E555F424013872
:100B4D00400B20E7087554FFF42401F5556190E83A
:100B5D00FAD3E813FC8852C3EF94036020EF20E032
:100B6D0007E82CF8ECFA617CE8282402F87AFEC339
:100B7D00EF940340088A54884E8C50619088548AB3
:100B8D004E8C50E56BC3335002646BF56B306002D5
:100B9D00619A753402D26043E680E52D54066026D5
:100BAD00A840A941C3E913F9E813F8C2AF53E67F92
:100BBD00759100C3E498F594E499F595759104D277
:100BCD006043E680D2AF22D26575440075200030B7
:100BDD006B03752040020BF3D26575440075204000
:100BED00306B03752000D2AF7801206722E52D54BC
:100BFD00066002C265C3E541940540137802940571
:100C0D0040087803940540027806306902780A207E
:100C1D006019E544601530690AC3E5339403400358
:100C2D00D53406D2AFD26C81C571A2D2AF0000C24D
:100C3D00AF206726E541C3FB940F40027B0FEB24E9
:100C4D000530730123306A02742820620123F930C4
:100C5D0069027982E58BC39940B50544E59BF4544F
:0E0C6D0040B5200281AF30690A08C3E8940A3E
:100C7B00400108811C20650261F3C26553E67F7554
:100C8B0091003067107594007595FE759104D260D4
:100C9B0043E68061F3AE40AF41C3E49EF594E49F1D
:100CAB00F5958196C3E5339402500261F3306502EA
:100CBB0061F3D80281C3811CC26C53E67F7591002E
:100CCB00855494855595759104854E56854F57D20D
:100CDB006043E680D2AFE52D54066008206A02051A
:100CEB0033020CFF306C0D206B0A20650715811544
:100CFB00810215652278003064053065027801E5C4
:100D0B003775F007A4F9E5F028F5F0E9A2F013A286
:100D1B00F113A2F213F537C394785003753778C3E8
:100D2B00E53795384008D266D290D291D292306096
:100D3B0002A139855056855157D26043E680222057
:100D4B007D11C2AF754302C294D293D2AF759F117E
:100D5B00020F19C2AF754302C294D295D2AF759FE1
:100D6B0011020F19307243207D20C2AF75430390DF
:100D7B00013D757E10D292C295306204C291A18D55
:100D8B00D294D2AF759F21020F19C2AF7543039056
:100D9B00013D757E10D290C293306204C291A1AD19
:100DAB00D294D2AF759F01020F19207D17C2AF7578
:100DBB004303900118D292306202C291D2AF759F59
:100DCB0021020F19C2AF754303900118D290306204
:100DDB0002C291D2AF759F01020F19207D11C2AFD4
:100DEB00754304C293D295D2AF759F01020F19C2FE
:100DFB00AF754304C295D293D2AF759F21020F19E1
:100E0B00307243207D20C2AF75430590012C757E57
:100E1B0008D291C294306204C290C129D293D2AF4E
:100E2B00759F11020F19C2AF75430590014E757E68
:100E3B0020D291C294306204C292C149D295D2AFF2
:100E4B00759F11020F19207D17C2AF7543059001D5
:100E5B000ED291306202C290D2AF759F11020F1960
:100E6B00C2AF754305900122D2913062EBC292D290
:100E7B00AF759F11020F19207D11C2AF754306C2CA
:100E8B0095D294D2AF759F21020F19C2AF7543064D
:100E9B00C293D294D2AF759F01020F1930724220C8
:100EAB007D20C2AF75430190014E757E20D290C25A
:100EBB0093306204C292C1C5D295D2AF759F010225
:100ECB000F19C2AF75430190012C757E08D292C2E7
:100EDB0095306204C290C1E5D293D2AF759F21E1E8
:100EEB0019207D16C2AF754301900122D29030625A
:100EFB0002C292D2AF759F01E119C2AF7543019047
:100F0B00010ED292306202C290D2AF759F21C2669F
:100F1B002290010C757E00D290D291D292C293C2D4
:100F2B0094C295C262227880760908760908760405
:100F3B000876FF0876030876FF087609087601081D
:100F4B007601087601788C76010876FF0876FF0823
:100F5B0076FF0876FF0876FF0876030876FF08769B
:100F6B00FF0876FF0876250876D008762808765095
:100F7B000876040876FF08760208760008767A0869
:100F8B0076FF08760108760108760008760322784A
:100F9B0087E6FFC2727888E6C394036008C27DE6D9
:100FAB0030E102D27DC27E7889E630E102D27EC387
:100FBB00EF94026008758E01D273020FCD758E000F
:100FCB00C273227880E6149000809378A4F678811F
:100FDB00E6149000809378A5F67886E61490008D41
:100FEB009378A6F6789CE67538FF75390CB4020633
:100FFB007538A075390AB4030675388275390578CA
:10100B00A3E61490009A93F569120F1C222278968E
:10101B00E6FA7897E6FB7888E6B40305C3EB940E03
:10102B00FB307F047A007BFFC3EB9AFCC3948250A6
:10103B00027C827575000575EC8575F0A4C3E5F02F
:10104B00947D40F222D27F111912059C7A007B000D
:10105B007C10120592E55F2AFA74003BFBDCF37CF3
:0F106B0004C3EB13FBEA13FADCF7FEC27F111983
:10107A0022E5EF20E6037520000520903FFFE520DA
:10108A00146006901DFF1460009304600375EF124C
:10109A0053D9BF7581C043FF8012058D75EF024396
:1010AA00B203E5B3240420E70DF521E5E320E006C9
:1010BA008521B343E301120F1C7580FF75A40075E7
:1010CA00F19175D47F75900775A53F75F2FF75D5B7
:1010DA000075A60175E241E4F8F6D8FD756B0112B8
:1010EA000F311215A778988676753001C2AF1205AE
:1010FA00A61205B612059C1205BD12059C1205C45E
:10110A0012059CC2AF78FA79FA308707D9FBD8F76B
:10111A00021C00120F9A120FCE1118111978988614
:10112A0076120F1C75885075891275C8247591043A
:10113A0075D84075A82275B80275E690759B8075BA
:10114A009D0075D10E75BC5875BB0675BA1175E848
:10115A008012058DD2AF12089A53DACF207E03434C
:10116A00DA20307E0343DA1043DA01C2D8C27112A0
:10117A0005A6D2617B037A0CE55E70077A0CDB0365
:10118A0002110D12059C20700302110DC270E55F59
:10119A00C3940240E1E52F541F856160F561B56093
:1011AA00D5DAD5C26153DACF207E0343DA20307E06
:1011BA000343DA10C2D8C27178A2E67008D274E585
:1011CA002F54E0F52FC2757529001205A130740954
:1011DA00C3E529940A4002D2751205927802307446
:1011EA00027800C3E55F9840F0C2AF1205B6120557
:1011FA00B61205B6D2AF1205A6754D007888E6B4C8
:10120A00030241E4120592788CE6C394015003026A
:10121A0012E4E530C3940150030212E4207435C38A
:10122A00E55F94FF50030212E4C2AF1205CBD2AFBE
:10123A001205A1C3E55F940150EFC2AF1205B612C1
:10124A0005971205B6D2AF1205A1C3E55F94FF4018
:10125A00E902174F7F02D27F11191205A1C2AFC24C
:10126A007F1119AE5FC3E55F947FD2AF4076120556
:10127A008DC2AF1205CBD2AFDFDC1150C3EE94059D
:10128A007897F61205A61215E91216D27F0AD27FAE
:10129A0011191205A1C2AFC27F1119AE5FC3E55F72
:1012AA00947FD2AF50E612058DC2AF1205B6120571
:1012BA00971205B6D2AFDFD61150EE24057896F60E
:1012CA001205A61215E91217011205A11119C3E593
:1012DA005F94FF5002412602174FC3E55F954D40C8
:1012EA0003855F4D1205A178017988E7B403027876
:1012FA0005C3E55F9840024106C2AF1205CB12054D
:10130A00CB1205CBD2AF1205A6753000E4F531F544
:10131A00320531E531F470390532789AE6781914D4
:10132A006012783214600D787D14600878FA1460BF
:10133A0003753200C3E53298401715327531B47817
:10134A00998676C2AF1205CBD2AF78988676120507
:10135A00A1120597E52A7005307402210D78012043
:10136A0074027806C3E55F9840A77888E6C39403B9
:10137A0060031205A1E52A700302110DC2AF120F14
:10138A001CE4F522F523F524F525F526F56AD2AFF6
:10139A007885E6C333F568E4F545F546F547F5483B
:1013AA00F549F573F52CF52DF53775730875BB10EE
:1013BA0012058D12089EE5E820ECFBA8BDA9BEE93E
:1013CA007001F888741208A275730875BB107887C3
:1013DA00E6FE7602120F9A7887EEF6C2AF7564FFC0
:1013EA0012093A852264852265852266D2AF752262
:1013FA000175240175250175260185636C756D01DA
:10140A007888E6B40307C27D307602D27DD268D2EC
:10141A0069753300120E82120EA712095A12096157
:10142A0012095A12096112095A021443C2AF120F61
:10143A009AD2AF75730075BB06120BE512069612A7
:10144A000D00120D4A120961120BD4306D031206F7
:10145A00F220670312083D306703120884120D0058
:0F146A00120D6F120961120BE5306D0312072787
:10147900120D00120DE6120961120BD4306D031220
:101489000785120D00120E0B120961120BE5306D62
:10149900031207E2120D00120E8212096112089E50
:1014A900120BD4120D00120EA71208A212096130F4
:1014B9006935206B3285676485676585636C756DF1
:1014C9000179187A0CC3E53399400FC269D26A8A47
:1014D900358567648567660214F0C3E55F9401404A
:1014E9000302144302156D306A1B206B18E535148D
:1014F9007004C26A8136F535C3E55F940140030281
:10150900144302156D753600C3E56278FA98505494
:10151900307404E52A604D7888E6B40317207D0508
:10152900207607A13D307602A13D206B07D26B855D
:101539006764818278F0306B058567647820C3E53C
:10154900419850028143306B1BC26BC27D307602D9
:10155900D27DD26A75351285676481430536E55FA8
:101569006002A170753600C2AF120F1C7887E6FEC3
:101579007602120F9A7887EEF6E4F522F523F52420
:10158900F525F526F568C268D2AF12058D120F1C34
:10159900307409C3E53694054002210D6116901A8D
:1015A9000D782012162BE520B4550CA312162BE545
:1015B90020B4AA030215C9120F311215E90215E860
:1015C900901A0378807B0A12162BA308DBF9901A6C
:1015D9000F788C7B1812162BA308DBF9901A272297
:1015E900C2AF12166A121644901A00740E121630FF
:1015F900A37404121630A37414121630901A0378C7
:10160900807B0A12162FA308DBF9901A0F788C7BBE
:101619001812162FA308DBF912167D12165B901A01
:101629002722E493F622E6438F01538FFD75EF02DB
:1016390075B7A575B7F1F0538FFE22438F02438F1B
:101649000175EF0275B7A575B7F1901A0DF0538FB3
:10165900FC22901A0D7455D130901A0E74AAD1300B
:10166900227A3079D07820901A40D12BE520F709D9
:10167900A3DAF7227A3079D0901A40E7D13009A35A
:10168900DAF922AB77A878BB01027980BB0202792B
:1016990081BB03027982BB04027984BB0502798686
:1016A900BB06027992BB07027987BB080279A3BB03
:1016B9000902799CBB0A027988BB0B027989E8F790
:1016C900227C051205A6DCFB22C2AF1205B6120563
:1016D900BD1205C41205CB1205971205B61205BD38
:1016E9001205C41205CB1205971205B61205BD12D3
:1016F90005C41205CBD2AF22C2AF1205CB1205C465
:101709001205BD1205B61205971205CB1205C412B2
:1017190005BD1205B61205971205CB1205C41205AF
:10172900BD1205B6D2AF22AE77AF78C2AF1205B6F9
:101739001205B61205B6120597DEF21205CB12058F
:1017490097DFF8D2AF22D1D2D1CAD1CA7577017544
:101759007801757900F1307C05AD5F1205A6C3EDFE
:10176900955F70F5C3E55F9401400AC3E55F94FF97
:10177900403202178BD18CB1E9D1D2C2AF75EF12C9
:10178900D1CADCD50579C3E5799403500280C6D165
:10179900CA0578E5771490009F93F808C3E578980F
:1017A900500280AED1CAD1CA0577C3E577940C50EF
:0F17B90002809C120F31B1E9C2AF75EF12D1CA95
:0319FD0002107B5A
:101A00000E0414090904FF03FF0901010155AA018D
:101A1000FFFFFFFFFF03FFFFFF25D0285004FF0259
:081A2000007AFF01010003FF41
:101A400023506F6C61726973546472333041232088
:101A500023424C48454C4923463333302320202031
:101A60002020202020202020202020202020202076
:101C0000C2AFC2D353D9BF7581C043B20343FF8073
:101C1000752438752503B1C975EF0275E24043F1AB
:101C20008053A47F75D400D2877DFA780379E67C4F
:101C300010752200752300901DD67B0675249875BB
:101C400025013087028142208708D8FBD9F9DCF7CB
:101C500081B4308708D8FBD9F9DCF781B4B189E4C5
:101C600093A3C39A6004DDC381B4DBDBB17B600264
:101C7000812B7B08E493FAA3B15CDBF87A30B15C8A
:101C8000752200752300B17BEAFCEBFDC3ED94FEE9
:101C9000400EB17B8A278B28ED30E0048A828B834B
:101CA000B17B7AC270D8C3ED94FE601350CEBD00F4
:101CB00025EC60097520007521FF0200008100A855
:101CC00027A9280809D804D90281D3B17FEA89AAB3
:101CD000F281C50D81A0C3ED94035049EDA2E092BD
:101CE000007AC5C3E5829400E583941C50902000DF
:101CF00010438F02438F0175B7A575B7F1F030001F
:101D00001FA827A9280809438F01538FFDD804D99C
:101D100002A12089AAE275B7A575B7F1F0A3A10DBC
:101D2000538FFC817C7AC1BD030CE493A3FAB140CC
:101D3000DCF8B138817C817EAA22AB23B15CEBFA5E
:101D4000EA6222752608C3E52313F523E52213F57D
:101D50002250066323A0632201D526EAB1C9B1C986
:101D600075260AEAF4200102D287300102C287B147
:101D7000C9C3134002C201D526EB22B17FEAFB2082
:101D80008702A17F308702A184752608AE24AF2583
:101D9000C3EF13FFEE13FEB1CDB1C9C3EA13308711
:101DA000024480FA30E703632201C3E52313F523DD
:101DB000E52213F52250066323A0632201D526D91C
:101DC000E52265236523F52222AE24AF250E0FDE22
:101DD000FEDFFCD20122424C48656C693437316326
:041DE000F3300601D5
:00000001FF
